:100000000C942A000C9445000C9445000C94450077
:100010000C9445000C9445000C9445000C9445004C
:100020000C9445000C9445000C9445000C9445003C
:100030000C9445000C9445000C9445000C9445002C
:100040000C9445000C9445000C9445000C9445001C
:100050000C94450011241FBECFE5D4E0DEBFCDBF18
:1000600010E0A0E6B0E0E6E2F1E002C005900D92FB
:10007000A036B107D9F710E0A0E6B0E001C01D92AC
:10008000A036B107E1F70C9468000C940000CF9300
:10009000DF93CDB7DEB722970FB6F894DEBF0FBE61
:1000A000CDBF1A82198289819A8125E78033920710
:1000B00034F489819A8101969A838983F4CF2296B8
:1000C0000FB6F894DEBF0FBECDBFDF91CF9108957C
:1000D000C8E5D4E0DEBFCDBF87E390E09D838C838D
:1000E00088E390E09F838E83EC81FD818FEF808396
:1000F00080E8898381E08A831B828B818430C0F70A
:100100000E944700EE81FF8199818A81892B809529
:1001100080838981869589838A81880F8A838B81F0
:060120008F5F8B83EACF24
:00000001FF
